:10000000200F00205D170000DF47000031170000BF
:1000100031170000311700003117000031170000C0
:100020000000000000000000000000008D1400002F
:1000300031170000000000003514000031170000E7
:100040000D1500000D1500000D1500000D15000028
:100050000D1500000D1500000D1500000D15000018
:100060000D1500000D1500000D1500000D15000008
:100070000D1500000D1500000D1500000D150000F8
:100080000D1500000D1500000D1500000D150000E8
:100090000D1500000D1500000D1500000D150000D8
:1000A0000D1500000D1500000D1500000D150000C8
:1000B0000D1500000D1500000D1500000D150000B8
:1000C0000D1500000D1500000D1500000D150000A8
:1000D0000D1500000D1500000D1500000D15000098
:1000E0000D1500000D1500000D1500000D15000088
:1000F0000D1500000D1500000D1500000D15000078
:100100000D1500000D1500000D1500000D15000067
:100110000D1500000D1500000D1500000D15000057
:100120000D1500000D1500000D1500000D15000047
:100130000D1500000D1500000D1500000D15000037
:100140000D1500000D1500000D1500000D15000027
:040150000D15000089
:1001540053B94AB9002908BF00281CBF4FF0FF312A
:100164004FF0FF3000F00CB8ADF1080C6DE904CE8F
:1001740000F008F8DDF804E0DDE9022304B070477C
:10018400704700BF2DE9F04F07468C460846099E8C
:1001940015463C461946002B40F0C5808242B2FA0F
:1001A40082F746D94FB1C7F1200E00FA07F3BD40DC
:1001B40024FA0EFEBC404EEA030C4FEA15481FFA1F
:1001C40085FE220CBCFBF8F908FB19C309FB0EFAE7
:1001D40042EA03439A4528D9EB1809F1FF3004D2C7
:1001E4009A4502D9A9F102002B44A3EB0A03A4B255
:1001F400B3FBF8F208FB123302FB0EFE44EA03449D
:10020400A64514D92C1902F1FF3303D2A64501D90E
:10021400931E2C44A4EB0E0443EA00401EB1FC40A0
:10022400002334607360BDE8F08F4846DDE7134671
:10023400F0E702B9FFDE87BB831A01214FEA154EAE
:10024400AAB2200CB3FBFEFC0EFB1C330CFB02F821
:1002540040EA0343984562D9EB180CF1FF3004D20D
:10026400984502D9ACF102002B44A3EB0803A4B2D5
:10027400B3FBFEFC0EFB1C330CFB02F244EA03440A
:10028400A2424ED92C190CF1FF3304D2A24202D956
:10029400ACF102032C44A41ABEE7C7F1200CBD4004
:1002A40000FA07F320FA0CF84FEA154E24FA0CFC76
:1002B400BC404CEA0302ABB2B8FBFEFC110C0EFBD3
:1002C4001C800CFB03F941EA0040814523D928181E
:1002D4000CF1FF3104D2814502D9ACF1020128446A
:1002E400A0EB090092B2B0FBFEFC0EFB1C000CFB61
:1002F40003F842EA004398450FD9EB180CF1FF329A
:1003040004D2984502D9ACF102022B44A3EB0803B2
:1003140042EA014192E76146E2E76246F6E7604657
:10032400A3E76346B7E7834205D90EB1C6E9007077
:100334000021084677E7B3FA83F181B9834201D3F8
:10034400BA420AD8BC1A60EB030301209C46002E73
:1003540067D0C6E9004C002165E70846F7E7C1F11C
:10036400200C8B4002FA01F522FA0CF420FA0CFB63
:1003740027FA0CF28F401C4300FA01F34FEA1449A8
:1003840013431FFA84FE1A0CBBFBF9F809FB18BBD4
:1003940008FB0EFA42EA0B4292453ED9A21808F134
:1003A400FF3004D2924502D9A8F102002244A2EB04
:1003B4000A029BB2B2FBF9F809FB182208FB0EFEF5
:1003C40043EA024296452AD9A21808F1FF3304D21F
:1003D400964502D9A8F10203224443EA0040A2EB65
:1003E4000E02A0FB05939A42CE46984602D306D14C
:1003F4004F4504D20138B9EB050E63EB040886B10E
:10040400B7EB0E0362EB080707FA0CFCCB40CF40B6
:100414004CEA0303C6E900379DE74046C7E7434675
:10042400DBE73146FFE6000038B5104C204604F007
:1004340094FDC8B12269A56813681C2143F0805358
:10044400136020462B680A4A984700280CDB4FF0BB
:10045400805120466B699847002805DB00214FF442
:10046400004003F01DFDF2E738BD00BFBC520000A0
:10047400010006000B6801330B60014B1B68184731
:1004840000000020014B1860704700BF00000020EE
:1004940007B50B46002102460191034801A900F06B
:1004A400E5F803B05DF804FB790400002DE9F84F8A
:1004B400B0F81890044619F0080893460DD00129A5
:1004C4000CBF49F0100949F02009A0F818908BF3EB
:1004D4001188BFF36F8FBDE8F88F09F0070902296F
:1004E40007D1204604F053F80028F0D00128238BCC
:1004F4004ED16769218B002F15DA256821F0070199
:10050400C4E9008841F0010121830026218B01F018
:10051400070ACA4502D0A368002B5AD10DB9002E90
:1005240071D0002356E001F007035A1F012A1ED898
:1005340021F00701062B256889B2C4E900880AD195
:100544003DB12A46638B126801339BB2002AFAD16B
:10055400638341F002012046218304F018F8064623
:100564000028D3D0238B43F020032383CDE7042B2F
:100574000CD121F0070189B22046218304F007F849
:1005840005460028C1D041F0200121830025BCE7A5
:10059400032809D1226923F00703166843F00603F0
:1005A400002523832F46B1E7042806D1226923F0CE
:1005B4000703566843F00403F2E7052806D12269CD
:1005C40023F00703966843F00503E9E700252E4668
:1005D400E8E7012341F0080121838BF31188BFF37D
:1005E4006F8FFBB985BB16B120461F49B0474FF04A
:1005F4002003EFF3118B83F31288BFF36F8F238BE8
:1006040023F008032383238BDA0625D5012123F065
:1006140010032383B4F8189009F0070900297FF424
:100624005EAF54E7A1680029DCD0D1F800903B46C6
:1006340052462046D1F804B0D847B9F1000FD1D0C2
:100644004946D9F80090F2E729463B4652462046EF
:100654002D6803F0B8FFC5E713F020011EBF23F097
:10066400200302212383D5E7F74500002DE9F04F4D
:100674008B4692461C46002591B002909AF80000E1
:1006840008B928465FE325280AF1010707D059462F
:10069400029B98470028C0F25683013512E21822C3
:1006A40000210AA804F0E5F89AF80130252B78D047
:1006B40000221046964694461646394617F8013BE2
:1006C4002B2B00F09D8000F29480202B00F09B8067
:1006D400232B00F09B802EB19DF8306046F0040679
:1006E4008DF83060BCF1000F05D09DF8306046F005
:1006F40008068DF83060BEF1000F05D09DF830601B
:1007040046F010068DF8306028B19DF8300040F0B6
:1007140020008DF830002AB19DF8302042F04002CC
:100724008DF830209DF8302002F04400442803D195
:100734006FF386128DF830209DF830202A2B42F07A
:1007440080028DF830207BD19DF831204B1C42F083
:1007540001028DF831201A782E2A0CBF01210021C4
:100764009DF8312061F341028DF8312074D15A781B
:100774002A2A6AD000210A260133184610F8012BD0
:10078400A2F13007092F40F28E809DF830200E919F
:10079400C2F3400040EAD17161F341028DF8302088
:1007A4005AE00AF102078DF833309DF83130D90749
:1007B40040F1498154F8049BB9F1000F07DA9DF820
:1007C4003020C9F1000942F004028DF830205A07A4
:1007D40040F1428154F8048BB8F1000F80F241815A
:1007E4009DF831306FF341038DF831304FF0FF380D
:1007F40037E12D2B0CD0302B7FF46DAF01225CE759
:100804004FF0010C59E74FF0010E56E7012054E771
:10081400012652E733460CFB0202303A1E4616F814
:10082400010BA0F13007092FF4D9994293D09DF818
:1008340030100D92D20F62F341018DF830108AE727
:100844000B4600224FF00A0CE8E79DF831200233F2
:1008540042F004028DF831201F4617F8012B6C2A50
:1008640041D025D8682A2BD06A2A46D04C2A4CD0AD
:100874001F4617F8012B9DF83130782A8DF8332064
:1008840000F2D980572A4DD8412A03D0453A022A8A
:1008940000F2D18004229DF8323062F302038DF815
:1008A400323001239EE006FB01210346303964E720
:1008B400742A26D07A2ADBD106229DF831300DE045
:1008C4005A78682A9DF8312006D1012161F3C602C5
:1008D4008DF831209F1CCCE71346022262F3C60335
:1008E4008DF83130C5E75A786C2A9DF8312001D152
:1008F4000421EBE713460322F0E705229DF831308B
:10090400ECE707229DF83130E8E7BDF8303023F4F6
:10091400F04323F0020343F4804343F00203ADF8B1
:100924003030A6E7A2F15801202900F2848001A00A
:1009340050F821F0FD0900003B0A00003B0A0000CA
:100944003B0A00003B0A00003B0A00003B0A00008F
:100954003B0A00003B0A0000990800003B0A000023
:10096400FD090000BD090000990800009908000075
:10097400990800003B0A0000BD0900003B0A000082
:100984003B0A00003B0A00003B0A0000050A000085
:10099400FD090000210A00003B0A00003B0A000098
:1009A400210A00003B0A0000FD0900003B0A000088
:1009B4003B0A0000FD09000001209DF8321003F0FD
:1009C400780360F30201402B8DF8321002BF9DF8CA
:1009D400301041F001018DF83010632A31D1003B11
:1009E40018BF01239DF83020C2F340010B4363F389
:1009F40041028DF83020D8E602209DF83210DEE75F
:100A040003219DF8322003F07803A3F1400061F341
:100A1400020243428DF832204341E3E703219DF86B
:100A2400322013F0780F61F3020214BF0123002374
:100A34008DF83220D6E79DF8303043F001038DF86D
:100A440030300023CEE79DF93020002AACBF4FF0B0
:100A5400FF39DDF83490BAE69B077FF5C7AEDDF8C1
:100A640038800023CDE90D339DF832309DF83110E4
:100A740003F00703012BC1F3C30138D1CB1E042BB0
:100A840022D8DFE803F003090921210054F8043BCC
:100A9400DA17CDE90A3206E0073424F00704F4E853
:100AA4000223CDE90A239DF8303013F0030656D013
:100AB4003B4652465946029803F064FE0028C0F2B1
:100AC40042810544BA46D9E554F8043B01294FEA6A
:100AD400E372CDE90A3205D19DF828300A93002348
:100AE4000B93E0E70229DED1BDF92830D0E7022BD1
:100AF40023D1CB1E042B13D8DFE803F0030A0A1218
:100B0400120000232268201D0A920B930446CAE7B0
:100B1400E01D20F00700F0E80223CDE90A23F5E701
:100B240054F8043B01290A934FF000030B93D3D0EC
:100B34000229B8D1BDF82830D0E7042B09D1E31D30
:100B440023F0070303F10804D3E90023CDE90A23C2
:100B5400A9E7032B04BF54F8043B0A93A3E79DF8C9
:100B640033007828AED8622822D825283FF48FADE8
:100B74005828A7D1DDE90A010DF1260300930CAA38
:100B840004AB03F0B9FD8246B8F1000F0DF1260065
:100B94000CDB9DF83020A0EB0A036FF38612984516
:100BA4008DF8302002D9A8EB03030D9380463DE075
:100BB4006338152886D801A252F820F0410C0000B1
:100BC400A50C0000C90A0000C90A0000C90A0000F7
:100BD400C90A0000A50C0000C90A0000C90A0000E7
:100BE400C90A0000C90A0000FF0C0000CD0C000077
:100BF400D10C0000C90A0000C90A0000190C000049
:100C0400C90A0000CD0C0000C90A0000C90A00008E
:100C1400CD0C0000B8F1000FDDF828A00ADB414636
:100C2400504603F012FE00260AEB0008BAF1000F4A
:100C34000CD147E7504603F001FEF4E700260A9B77
:100C44000DF1100A8DF810300DF11108A8EB0A030C
:100C540006B101339DF83220D00668D5023352061E
:100C64000D9948BF0E9A0B4448BF9B18B9F1000F69
:100C740076DD9DF83020A9EB0309C2F380030393CA
:100C840053076DD4500661D546B159463046029B90
:100C94009847002857DB039B01351E46302356E056
:100CA4001E070FD413F0100618BF2026DDE90A230F
:100CB400002BBFF65FAF524263EB43032D26CDE911
:100CC4000A2357E72B26F1E7002653E70A9840B397
:100CD4000DF126030093002104AB0CAA03F00CFDD4
:100CE400BDF83230824603F0EF0343F4F04343F09F
:100CF40010030026ADF8323046E70A9B07293FF679
:100D0400E1AEDFE801F00C04060C08080C0C1D70C1
:100D1400D8E61D80D6E6EA17C3E90052D2E61D6084
:100D2400D0E6DFF8C8A006460AF105088EE71107E9
:100D340048BF013393E7184603935946029B9847EB
:100D44000028039B04DA11B0BDE8F08F20234D4442
:100D54004A46002AA5EB090109F1FF39EBDC0D46EF
:100D640036B159463046029B98470028EBDB0135E3
:100D74009DF83230D90601D41A0706D559463020D9
:100D8400029B98470028DEDB01359DF83230DB06F4
:100D940007D559469DF83300029B98470028D2DBBB
:100DA40001350D9E2E44731B002B16DC4346524620
:100DB4005946029803F0E6FC0028C4DB0544A94424
:100DC400A9EB0503002B7FF77DAE59462020029B3B
:100DD40098470028B7DB0135F2E759463020029BDB
:100DE40098470028AFDB0135DDE700BF2C57000032
:100DF40008B54FF02002EFF3118382F31288BFF39A
:100E04006F8F00F0D9FC034803F0B4FB00F08AFABA
:100E1400FCE700BF32570000054B03EB8000D0F81D
:100E2400003223F0E04343F04053C0F800327047EF
:100E34000025845010B54FF02003EFF3118483F3A1
:100E44001288BFF36F8F01220C4B0D49C3F80025A4
:100E540002230020C1F8D036FFF7DEFF1046FFF76B
:100E6400DBFFC1F80427C1F80429C1F8002B84F37F
:100E74001188BFF36F8F002010BD00BF0010005019
:100E84000040005048B1054B1A68054BB2FBF3F221
:100E9400044B504343F001031847704740000020BF
:100EA40040420F0050550000062807D10122044B90
:100EB400C3F80025BFF34F8F20BFFDE7704700BF85
:100EC400004000502DE9F84305464FF02003EFF3AE
:100ED400118683F31288BFF36F8F0E4B1C689CB18D
:100EE4004FF00C090C4FDFF83480D4E90132002DA7
:100EF40008BF13462BB198F8142009FB02F2B85C22
:100F040098472468002CF0D186F31188BFF36F8FC3
:100F1400BDE8F883B8020020C002002008090020C0
:100F24000123420900F01F0003FA00F0C043054BFF
:100F340003EB8203D3E8EF2F0240C3E8E12F00293B
:100F4400F8D17047CC020020012238B5174B1C7D24
:100F540004F01F039A40D043154B610903EB81034E
:100F6400D3E8EF1F01EA0005C3E8EC5FBCF1000F12
:100F7400F6D1114213D00F4B0F4D8BB10C236343A9
:100F8400EA185178E85C03F014FC0020FFF79AFF9C
:100F94000C235C4300232A192B51C2E9013338BDC9
:100FA40083F31188BFF36F8FEFE700BF08090020B8
:100FB400D0020020B7470000C00200202DE9F8430A
:100FC4002F4B07461C7D4FEA54184FEA88082D4BD7
:100FD4004344D3E8AF3F04F01F0943FA09F313F085
:100FE400010F294E0AD10146204600F063F828B1CA
:100FF40007C80C2303FB046383E807000C23634343
:10100400F55CF2182DB92046FFF78AFF2846BDE8A3
:10101400F8837B1C0FD04FF400450021D2F808C0A0
:101024001A480023ECFB0501194AFFF791F8012146
:10103400381A04F0E3F802F0B3FC0120FFF742FF92
:10104400012303FA09F9134B9844D8E8EF3F43EA24
:101054000903C8E8E23F002AF7D10F4B33B10C2350
:101064006343F2185178F05CFFF71EFFFFF76CFF43
:101074002046FFF755FF02F063FE0120C7E700BFDB
:1010840008090020CC020020C00200203F420F00CB
:1010940040420F00D0020020AD0E0000044B03EBD1
:1010A4008000D0E8AF0F003818BF0120704700BFA0
:1010B400D40200202DE9F04F85B00F4603A900F0BB
:1010C40047F84FF0000B441EDFF87880DFF878A073
:1010D40024B2631C04D10026304605B0BDE8F08F6D
:1010E400039A04EB440312F8230002EB8306FFF790
:1010F400D5FF054610BB4FF40049C4462946706825
:101104005246E0FB09C15B466046FFF721F8C4463E
:1011140029460190B0685B46E0FB09C1524660462F
:10112400FFF716F8094B1B68591C01D0834205D9F7
:101134007A1CD1D0019B1844B842CDD9013C24B2C9
:10114400C7E700BF3F420F0040420F0004000020E9
:1011540008B9024B0B600020704700BF58550000CF
:10116400014803F0BDB800BF5855000010B504464F
:1011740018B90D4B0D485B689847616808290DD074
:1011840031F004030AD011F0020108D021460848C6
:1011940003F027FF002323600023636010BD1422A3
:1011A400206803F066FBF7E7CC0000205B570000E3
:1011B400F002002008B540B34368042B0BD0082B81
:1011C40016D003B300684FF0FF324FF0FF3302F044
:1011D4008DFA58B115E001220368D3E8EF1F002906
:1011E40003D1C3E8E02F0028F7D10AD1002008BDBD
:1011F4000368074A1B7803F5807352F82330002BE9
:10120400F4D00448F3E70448F1E76FF4E040EEE774
:1012140000000350E98FFFFFEA8FFFFF08B508B312
:101224004368042B07D0082B13D0F3B1006802F0F5
:10123400D5FA00200CE000220368D3E8EF1F01294F
:1012440003D1C3E8E02F0028F7D1094808BF1046AE
:1012540008BD036800201B78064A03F5807342F832
:101264002300F5E76FF4E040F2E70348F0E700BF3E
:10127400E98FFFFF00000350EA8FFFFF10B504461B
:1012840018B9164B16485B6898476368042B23D03B
:10129400082B21D0CBB92368BBB94FF0FF324FF0F4
:1012A400FF3321460F4802F04BF908B923681BB9F4
:1012B4000A4B0D485B68984714220021206803F00C
:1012C400D8FA636843F002036360206803F0C7FE42
:1012D400636843F00103636010BD00BFCC000020CD
:1012E4005B570000F00200208157000008B5064952
:1012F40040231422054803F059FEBDE80840044980
:10130400044803F04FB800BF0C030020F002002093
:101314007055000060550000014910220A607047B2
:1013240010ED00E072B6404080F31188BFF36F8F78
:10133400BFF34F8F30BF62B6BFF36F8F704700BFEC
:1013440072B6494081F3118820BF80F3118862B6D8
:10135400704700BF43B2002B08DB012200F01F00DE
:1013640002FA00F0024A5B0942F82300704700BF0A
:1013740000E100E0054B420953F82220012300F06C
:101384001F0003FA00F01040704700BF00E100E0C6
:1013940043B2002B01F10101ACBF03F16043064BE2
:1013A4004FEA4111C9B2ABBF03F5614300F00F002E
:1013B40083F800131954704714ED00E030BFFFF7B1
:1013C400FDBF00BF0B4A08B50B4B22F07F029A60A9
:1013D400BFF34F8FBFF36F8FD3F8882022F47002CE
:1013E400C3F8882001F0E0FF02F0CCFD00F0A8F97A
:1013F40002F01AF80000000000ED00E0094A0A4972
:10140400936809685867996708494B6843F08053A3
:101414004B60002383F31188BFF36F8F9368986F39
:10142400704700BF080900209C56000000ED00E052
:1014340013498A684FF030001044EFF3098C80E8B8
:10144400F01F202080F31288BFF36F8F0D4F4FF0F1
:101454000066CA698A603E60506F0023536780F358
:10146400118802F1300090E8F01F8CF3098802F132
:10147400000004B503F0B8F9BDE80440704700006B
:101484000809002004ED00E01EF0040F0CBFEFF388
:101494000880EFF30980816911F8021C0229FFD04A
:1014A40001B503F092F901BD42F8203C009B0B49C1
:1014B40042F81C3C019B21F0010142F8183C029BBC
:1014C40042F8081C42F8143C4FF0807342F8043C84
:1014D4000023203A02654367704700BFE9460000D5
:1014E400084B9860436E83F30B88104681F3098898
:1014F400002163B681F31188BFF36F8F00220023AC
:1015040003F0F0F80809002001B572B60B4A90699F
:1015140000281EBF0021916103F092FD62B6EFF333
:101524000580A0F110004FEAC0000549014409C933
:101534009847BDE801400349084700000809002016
:10154400045300004D150000044B9968D869884283
:1015540003D003494FF080520A6070470809002005
:1015640004ED00E0094B9A6A9A6A986A9A6A9A6A40
:101574009A6A9A6A9A6A10F480106FEA02426FEAD1
:10158400124218BF02209A62704700BF00ED00E0CB
:101594000D4B9A6A9A6A9A6A920508D59A6B9A6A66
:1015A400120404D518B19A6A22F400429A62002007
:1015B400054B9A6A9A6AD20558BF9A6A9A6A42F4A3
:1015C4007F429A620870704700ED00E0124B9A6AFD
:1015D4009A6A9A6A920708D55A6B9A6A120604D5CF
:1015E40018B19A6A22F080029A620B4B9A6A9A6A3C
:1015F4009A6AD0064FF0000058BF9A6A9A6A920617
:1016040042BF5A6A22F400525A62034A936A43F070
:10161400FF0393620870704700ED00E070B53C4B27
:101624000E465B6800258AB0C3F3080385F311886E
:10163400BFF36F8F02F07F41B1F17F4F11D102F000
:101644000C0108290DD0110701D4064601250022FA
:10165400033B8DF80720032B52D8DFE803F004493D
:101664004D462E46F3E72A4BDC6A14F0020447D1B8
:10167400DA6A002A14DBDA6A520011D5B26932F848
:10168400021C4DF60272914209D093F82820FAB157
:1016940001200DF10701FFF799FF044600E03468CB
:1016A4009DF8073093B92022314602A803F0D6F8FA
:1016B400099B3DB3C3F3080222B96FEA53236FEACF
:1016C40043230993204602A903F07DF80AB070BDB4
:1016D40093F829202AB101200DF10701FFF758FFE3
:1016E400DBE75B8D9BB2002BDAD0FFF73BFFD4E73F
:1016F40000200DF10701CEE700200DF10701EDE711
:101704000024CDE723F4FF7323F00103D9E700BFDE
:1017140000ED00E0044B5A6942F010025A615A6924
:1017240042F480625A61704700ED00E0EFF30880F4
:10173400EFF3098101B57246FFF770FF01BD00BFE9
:10174400002320210348C2180133452B82F80013DB
:10175400F9D1704700E100E0002080F31488BFF362
:101764006F8F002080F30A8880F30B8803F06AFDF2
:1017740000200E490860BFF34F8F0D4880F308889E
:1017840000F03EF8202080F311880A484FF40061ED
:10179400401880F30988EFF314800221084380F392
:1017A4001488BFF36F8FFFF70DFE000094ED00E087
:1017B400200F002060100020BFF34F8F0549064B17
:1017C400CA6802F4E0621343CB60BFF34F8F00BFDB
:1017D400FDE700BF00ED00E00400FA050023184611
:1017E4000649D1F89020C2F30722934200D17047F2
:1017F400C1F89830C1F8A0000133F6E700ED00E02D
:1018040010B572B6002484F31388FFF7E7FF23466C
:101814004FF0FF300B4A03F120010133102B42F843
:101824002100F8D100234FF0FF3003F160010133B0
:10183400102B42F82100F8D162B6BFF34F8FBFF3EB
:101844006F8F10BD00E100E0084B9B6883420BD111
:10185400EFF3058343B1064B5A6842F080525A6055
:101864005A6A22F400425A6202F03ABB0809002084
:1018740000ED00E01FB5094C094A2346012109483F
:1018840000F0F2F800230393074B0121E41A01A8A6
:101894000193029400F0F2F804B010BD0000072098
:1018A40000000020845500009001002010B50B6852
:1018B4000C7A23F01F0204F01F031A43CB68640957
:1018C40023F01F03054943EA440343F00103C1F82D
:1018D4009800C1F89C20C1F8A03010BD00ED00E0D4
:1018E4002DE9F04F0F46144606464FF00008524DBE
:1018F40085B0B84509DAD6F80490B9F1000F3AD0AA
:10190400B9F11F0F05D86FF01504204605B0BDE8E6
:10191400F08F19F01F0FF6D1D6F800A01AF01F0FA0
:10192400F1D1504602F064FF834609EB0A00013806
:1019340002F05EFF8345E6D11BF1160FE3D05C4550
:10194400E1DDC5F898B0D5F89C10C5F898B0D5F885
:10195400A03021F01F0143F01F0AD6E900321A44D7
:10196400994202F1FF391ED1CA4508D131465FFAC6
:101974008BF002F046FF08F101080C36B9E7314656
:10198400C5F898B0D5F89C3022F01F0203F01F036D
:101994001A43C5F89C20E0B202F033FF10F1160F91
:1019A400B1D0441CE7E7013BCA45E0B223F01F0372
:1019B400C5F898B008D1D5F8A020314602F01F022E
:1019C4001343C5F8A030E7E7D5F8A01001F01F01D4
:1019D4000B43C5F8A030314602F013FF10F1160F87
:1019E40091D0C5F898B0D5F89C209DF808300AF13C
:1019F400FF3A62F304038DF80830D5F8A0309DF85F
:101A040008205B0863F347128DF80820D6E90032FA
:101A14001344009323F01F03411C5344A3EB090315
:101A2400C8B223F01F03072803933FF66CAF69463F
:101A3400FFF73CFFB5E700BF00ED00E00522044BD3
:101A4400C3F89420BFF34F8FBFF36F8F704700BF6D
:101A540000ED00E0BFF35F8F0022024BC3F8942037
:101A6400704700BF00ED00E010B5034C2278FFF78B
:101A740037FF207010BD00BF180B00202DE9F74F71
:101A8400294D8A4606464FF00008AB46274FD045FD
:101A94001BDAD6F80490B9F1000F3FD0316808463C
:101AA400019102F0A5FE0199044609EB01000138F9
:101AB40002F09EFE84424FF014021D4B08D06FF0DA
:101AC400150302FB08F84BF8083003B0BDE8F08FAB
:101AD40014F1160F2C60F8D01978A142F5DD02FB41
:101AE40008B0C7F89840C7F89840D7F89C4000F170
:101AF4000801007B64F304000871D7F8A0000C7996
:101B0400400860F347140C71D7F89C1021F01F01B2
:101B14006960D7F8A01021F01F01296108F10108BC
:101B240014350C36B3E700BF0C08002000ED00E0CC
:101B3400180B002038B50E4D2C68082C15D8002041
:101B4400FFF788FF0B4B0C4AC3F8C020844205D131
:101B54000A4B00201C70FFF771FF38BD696801EB68
:101B64000011FFF7A3FE0130F0E74FF0FF30F4E778
:101B74009055000000ED00E0AAFF4400180B00207F
:101B8400014B1860704700BF28000020084B70B557
:101B9400C31A0D4607499B10044659434022064880
:101BA40002F08FFE2B4601462046BDE870401847E0
:101BB40030080020B76DDBB6A4520000402373B593
:101BC4000B4C0093041B0B460D460A49A4106143B9
:101BD4000646094A094802F0A0FE011E05DA30460D
:101BE4002B4602B0BDE87040184702B070BD00BF7C
:101BF40030080020B76DDBB68F490000A452000006
:101C04002DE9F8430022012106460520FFF7C0FB19
:101C1400114800F0BFFF114B984219D103F0D2F8DC
:101C240000244FF01C080C27DFF83490356949462E
:101C340008FB045002F0FAFC002807DB012307FB31
:101C440004551C44042CAB67F0D10020BDE8F88394
:101C54006FF00400FAE700BF9D1C00000000AD0B0C
:101C6400F055000001460C2300224B43084870B590
:101C7400C4187833D4E91C561844226702F00EFEC7
:101C84002DB132462B46BDE870400248184770BD5E
:101C940030080020A4520000052811D8DFE800F025
:101CA400030E10100C0A074B986F10F0070007D1B1
:101CB400FFF7D8BF0220FBE70320F9E70120F7E78D
:101CC400704700BF3008002008B54FF02003EFF341
:101CD400118183F31288BFF36F8F124A136843F0A4
:101CE400020013F0010310600CD04FF05022D2F820
:101CF4000C34D2F80C2413F0010303D00A4802F088
:101D0400CDFD012381F31188BFF36F8F23B1BDE8AB
:101D140008400020FFF7A6BF0120BDE8084003F0FB
:101D240063B800BFD0080020A80800201FB5002217
:101D34000123CDE902236B46084ACDF800D0CDF843
:101D440004D002F01BFE002805DB4FF48042002380
:101D5400684601F0A5FD05B05DF804FBC549000027
:101D6400074BD3E8EF2F22F00201C3E8E01F00285D
:101D7400F7D1D30702D4012003F096B8704700BF0F
:101D8400D00800202DE9F041012207463749D1E867
:101D9400EF3FC1E8E02F0028F9D133B93449354881
:101DA4004B60CB608A6002F054FC7B1E012B2FD861
:101DB400012F07D14FF05023D3F81C3403F0030351
:101DC400022B25D003F036F9044618B92A4B1B78A8
:101DD400002B44D14FF02003EFF3118683F31288D4
:101DE400BFF36F8F01244FF05025DFF89080D5F8B2
:101DF4001834D5F81824D2030CD503F00303022BAE
:101E040001D0012F06D124B386F31188BFF36F8F5D
:101E1400BDE8F081C4B13046FFF792FAD5F8183521
:101E2400DBB2012BE3D1D5F80421002ADFD0002254
:101E3400C5F80421D5F804210222C5F8182520226A
:101E4400C8F88021AB60D2E70021212002F028F8F5
:101E5400E4E74FF050230222C3F80423D8E74FF0FD
:101E6400502302220646C3F80823BCE7D408002006
:101E7400200800204C080020190B002000E100E09D
:101E840008B50848084B186003F067F838B10748EC
:101E9400FFF776FE0548FEF7F5FA002008BD6FF05F
:101EA4001200FBE7EC520000D8080020B51E000029
:101EB4000A2838B50446074D04D1286883680D21E3
:101EC4005B68984728688368E1B25B689847204656
:101ED40038BD00BFD808002030B5406801F01F05A8
:101EE400047BB2F5001F45EA441585B04FF00004A9
:101EF40004D1284601F0FCF8002031E0B2F5800F4F
:101F0400CDE902442ED1B3F1007F0CBF0423052395
:101F14008DF80830836823FA01F1C9072ED4B2F191
:101F2400A07F2BD11E4A1F486909012908BF024618
:101F340005F01F03803352F82330DB071ED40DF164
:101F440007042146284601F039F8174B984214D16A
:101F5400204601F081F8154B98420ED06FF00B002B
:101F640005B030BDB3F1C06F05D0B3F1007F0CBF35
:101F740002230123CCE70323CAE703940023284662
:101F8400194602AA00F0F4FE084B984204D101213C
:101F9400284601F067F8AFE76FF00400E0E700BF00
:101FA40000258450002884500400AD0B0000AD0BC4
:101FB40010B501F041F8044668B901F015F8084B72
:101FC40098420AD12146074800F0F2FF2246052133
:101FD4000D20FFF7DDF9002010BD6FF00400FBE7D2
:101FE4000000AD0BED1F00004209034670B502D09E
:101FF400012A15D070BD0B4E326951680029F9D001
:10200400012503F01F030C689D408A682A4002D012
:1020140030464B689847002CECD021462468F4E7FE
:10202400014EE9E7BC520000D45200002DE9F04310
:10203400476801F01F053B7B0E46144685B045EA10
:102044004315CAB902A9284600F0B8FF0446284639
:1020540001F076F8494B984204D06FF0040005B0C3
:10206400BDE8F083844205D19DF8080000F0EEFF3E
:10207400A042F2D10020F2E74FF000090DF1030174
:102084003046CDE9029900F099FF4B468046494617
:10209400284602AA00F06CFE384B984202D06FF03A
:1020A4001500DCE7804503D19DF8030000F0CEFF66
:1020B400A3034FD540F2066340F206222340934225
:1020C4003AD00CD8062B15D004D89BB1022BE6D1FC
:1020D40004230FE0B3F5007FE1D101230AE040F2CD
:1020E400024293422AD0B3F5C06F29D0B3F5806F72
:1020F400D5D102238DF8043084F48033C3F3004334
:10210400E0068DF805304CBF0323C4F340132103CC
:102114008DF8063016D501217B6801FA06F69E601B
:102124000022284601A900F0CFFE144B984214BFA8
:102134006FF01500002092E70723DBE70523D9E7BA
:102144000323D7E7620341BF01217B6801FA06F646
:10215400DE60E5E7E3064FF000034CBF0324C4F35D
:1021640040141A46284601A98DF8044000F000FEE8
:10217400024B98423FF47EAF91E700BF0000AD0BE5
:10218400F0B54B79012B28D0032B23D110278B7961
:10219400032B1FD1CD790DB1012D1BD10A79012A51
:1021A4001DD0022A1FD0AAB914460B684668B3F59D
:1021B400164F36686ED033D8B3F5165F6DD01CD881
:1021C400B3F5966F6BD010D8B3F5967F6AD0B3F59C
:1021D400167F6AD06FF085005BE00027D7E74FF4E5
:1021E40080740E22E1E70024FBE7B3F5166F5FD09D
:1021F400B3F5965FEED1394B3EE0B3F5E14F5AD0DB
:1022040007D8B3F5615F58D0B3F5964FE2D1344B9C
:1022140032E047F6122C6345DCD14FF400032BE087
:10222400B3F5613F4BD013D8B3F5963F4AD009D8E4
:102234004DF6C02C634547D0B3F5614FCAD14FF476
:102244006B0319E0B3F5E13FC4D14FF0EB7313E036
:10225400B3F5612F3BD009D8DFF888C0634539D086
:10226400B3F5E12FB6D14FF0E86305E0DFF878C0AD
:102274006345AFD14FF0805300692C433A43C6F80D
:1022840024352243031DC6F86C2503C983E80300E3
:102294000020F0BD4FF41D03EEE7144BECE74FF4C0
:1022A4009E23E9E74FF4A033E6E74FF41C33E3E75A
:1022B4004FF41D23E0E70E4BDEE70E4BDCE74FF057
:1022C4006C73D9E70C4BD7E74FF46503D4E74FF0B1
:1022D4007063D1E74FF08063CEE700BF00B0130016
:1022E40000A04E0090D0030040420F000050270091
:1022F40000C0750000F03A0000903A012DE9F74360
:102304000746002201210820FFF742F80820FFF7C2
:1023140021F80021D7F804803E69D8F80040D8F8A5
:102324000C90C4F800154846376001AA02F001FC7D
:10233400051E4FDB019BD9F800201979186802F0BB
:1023440015FC051E46DB3846311DFFF719FF05460F
:1023540000283FD1D8F80430990712D506F11200AD
:1023640000F080FC1F4B984238D1B27C42F000430D
:10237400C4F8A031C4F88C30012393401A4AC2F83F
:1023840004350823C4F8003598F808305BB9C4F85C
:102394001031D4F8103106F11103C4F83435012397
:1023A400C4F838352360D8F8043010369A075CBF77
:1023B4004FF48072C4F80423DB0644BF4FF4800357
:1023C400C4F804330023C4F84465C4F84835012331
:1023D400A360E360284603B0BDE8F0836FF0040512
:1023E400F8E700BF0000AD0B00700150F8B50546DA
:1023F4000F46066902F01EFE10B92C4B1B7883B9F8
:102404004FF02003EFF3118483F31288BFF36F8F2F
:10241400686802F044FB28BB84F31188BFF36F8F14
:10242400EEE76424686802F03AFB70B9012002F018
:102434004CFC013CF6D10021212001F031FDF0E7F4
:1024440084F31188BFF36F8FF5E74FF02003EFF3A8
:10245400118483F31288BFF36F8F686802F01FFB47
:102464000028EDD0012206F8107F69680B68C3F8D4
:102474004465C3F848250022C3F82021D3F820017D
:10248400C3F85821D3F858214A68D20641BF08221C
:10249400C3F800254FF48002C3F8042301229A6094
:1024A40084F31188BFF36F8FF8BD00BF190B0020B0
:1024B4000123834010B5DC430D4AD2E8EF1F01EA43
:1024C400040CC2E8EECFBEF1000FF6D14FF4803217
:1024D40002FA00F002F15022C2F80803BFF35F8F42
:1024E400BFF36F8F0B4214BF0120002010BD00BF4B
:1024F400F80800201949F8B5044622F07F45086819
:10250400C1E90023A5F50013101AB3F5400F22D238
:10251400134B1B681A0A1B065E19124B42F1000783
:10252400C3E90067012601F00BFEA30003F1502369
:1025340003F58033D3F84025AA420BD11EB94FF4DA
:102544000002C3F840254FF48030074B00FA04F42E
:10255400C3F84443F8BD0026E5E700BFA801002006
:10256400FC0800209001002000500150E1B101233B
:102574000E4A8340D2E8EF1F1943C2E8EC1FBCF1B6
:10258400000FF7D14FF48033094A8340C2F8043373
:10259400084BD3E8AF3F23FA00F0C30742BF4FF420
:1025A4000012054BC3F80021704700BFF808002053
:1025B40000500150F408002000E100E00D4B1868C1
:1025C400010A0006BFF35F8F0B4BD3F804351818CC
:1025D40041F10001B3F5801F0AD2084BD3E900236F
:1025E400904271EB030303D210F1807041F10001BA
:1025F400704700BFFC0800200050015090010020EB
:102604002DE9F04F85B0164698460546FFF750FF72
:102614000090FFF7D3FFB04271EB080376D2434B2F
:10262400301A68EB0101984271F100037BD2404BF0
:1026340003EB0513D3E902ABD84508BF564550D088
:102644004FF4803326F07F4214464FEA850905F1A2
:10265400500709F15029BF00AB4009F58039BFB2DA
:1026640007F150270193D9F84005324B07F580371D
:10267400D3F80415401A20F07F4021F07F4C012844
:10268400C9F840C507D1CDE90221132002F0D4FDD9
:10269400DDE90221274B01F1020CA4EB0C0020F030
:1026A4007F40B0F5000F88BF64460020386038686A
:1026B4000198C3F8440324F07F40C9F84005D3F8D7
:1026C4000405814206D0201A023820F07F40B0F57C
:1026D400000F19D8A41A24F07F4414EB060A48F119
:1026E400000B002412490E982B0101EB0512C8506F
:1026F400C2E902AB0F9B536028460099FFF736FFEF
:10270400204605B0BDE8F08F2046B1E701230A4A10
:10271400AB40D2E8EF1F1943C2E8E01F0028F8D10C
:10272400B246C346DDE76FF01504E5E7010000019A
:102734009801002000500150F408002073B50024D3
:102744004FF0FF304FF0FF31164D174BC5F80845D9
:10275400C3E902014FF4803302264FF40012C5F896
:102764000433124B0121C5F804631520C3F88021FA
:102774002246FEF70DFE1520FEF7ECFD01230C4A60
:10278400AB602B6013600B4B0B4A00932046002375
:102794000194FFF735FF3046FFF7F4FA204602B004
:1027A40070BD00BF005001509801002000E100E01E
:1027B400F8080020F9240000FFFF7F00354B2DE9C5
:1027C400F743D3F8042391070BD5D3F8042142B17E
:1027D4000022C3F80421304AD3F8043113680133CA
:1027E40013604FF02003EFF3118183F31288BFF3DA
:1027F4006F8F284BD3F80423D2030ED5274AD2E88F
:10280400EF0F20F00104C2E8E54F002DF7D10028B6
:1028140037D1D3F84021002A33D1002381F3118822
:10282400BFF36F8F53B3FFF7C9FE4FF02003EFF3ED
:10283400118783F31288BFF36F8F194BD3E90245D5
:10284400A04271EB05024FF0000221D3D3E9001638
:102854004FF0FF384FF0FF391A604FF48032C3E96C
:1028640002890C4BC3F8482387F31188BFF36F8F99
:1028740021B122462B4600200096884703B0BDE8CC
:10288400F0830022C3F84021D3F840310123C5E787
:102894001146E9E700500150FC080020F40800202C
:1028A40098010020431C13B520D0012820DDB0F589
:1028B400000F1FDA441EFFF781FE0F4BD3E900130C
:1028C400401AB0F5000F28BF0024013002190B484C
:1028D400824228BF02460020521809490190009103
:1028E40043F10003FFF78CFE02B010BD0348E1E79B
:1028F4000024E0E7014CDEE7A8010020FFFF7F0091
:10290400F924000008B5FFF759FE024B1B68C01AF2
:1029140008BD00BFA8010020054A064B00F01F01B6
:102924004009012808BF134601228A40DA60704733
:10293400002884500025845000F4805370B5002B87
:102944000F4E0EBF15460125002110F0200F0D4B30
:1029540018BF334600F01F04C0F3811203EB840355
:1029640000F47060D3F8004240EA82020A4304F0A3
:10297400E04442EA45022243C3F8002270BD00BF8E
:102984000028845000258450054A064B00F01F019E
:102994004009012808BF134601228A409A60704703
:1029A40000288450002584504FF47F03D3F830214D
:1029B400D3F83431072A05D1023B032B02D8024A4B
:1029C400D05C704700207047D85700004FF0502368
:1029D400D3F85825034B02F00302D340024A136094
:1029E400704700BF0020A1074000002008B5FFF792
:1029F400DBFF58B13F4BD3F8202A3AB90D21C3F875
:102A0400201A0121C3F81C19C3F81C290022D30081
:102A140003F57F03D3F80013013107D0D3F8001373
:102A24000132D3F80433202A0B60F0D1FFF7BCFF46
:102A3400002857D1FFF7B8FF40B12F4B2F4AC3F8F6
:102A440030254FF050230122C3F858254FF47F035B
:102A5400D3F83021D3F83431072A09D1023B032BB0
:102A640006D8274AD35C1BB10022264BC3F84C2559
:102A7400FFF79AFF50B14FF05023D3F80024D10749
:102A840042BF0022C3F81421C3F818214FF47F0376
:102A9400D3F83021D3F83431072A09D14FF0502329
:102AA400D3F80024D20744BF6FF00102C3F8002416
:102AB400FFF77AFF18B165220E4BC3F80C27124AB0
:102AC400D2F88C3043F44063C2F88C300F4A104B78
:102AD4001168C3F84415D269C3F84C25BDE8084011
:102AE400FFF774BF2922034BC3F80C270322C3F852
:102AF4003C279FE700400050009003504400EFBE85
:102B0400DC5700000020035000ED00E00080FF00CF
:102B14000060005070B501250268B2FA82F3C3F177
:102B24001F035E1CDCB210D005FA03F322EA030390
:102B3400D0E8EF6F964204D1C0E8EC3FBCF1000F3F
:102B4400F6D1E9D102480C7070BD0248FCE700BF21
:102B54000000AD0B0200AD0B036810B5CB40DB07E2
:102B640011D4012303FA01F1036841EA0302D0E816
:102B7400EF4F9C4204D1C0E8EC2FBCF1000FF6D11A
:102B8400F2D1024810BD0248FCE700BF0000AD0BC3
:102B94000400AD0B044B1A7922B9012218601A7192
:102BA4000248704702487047000900200000AD0B3E
:102BB4000C00AD0B4FF05023D3F8002110B552B1E7
:102BC4000020C3F80001D3F800210122C3F8082330
:102BD400234B1B6898474FF05023D3F804218AB144
:102BE4000022C3F80421D3F80421D3F81824D3F81D
:102BF400181402F00302012A4FF0020128D1C3F88D
:102C040018159A604FF05023D3F8202162B10022A6
:102C1400C3F82021D3F820214FF48072C3F808238D
:102C24000F4B04201B6898474FF05023D3F82421FE
:102C3400AAB1BDE810400022C3F82421D3F824210E
:102C44004FF40072C3F80823054B05201B6818478E
:102C5400C3F80813024B01201B689847D2E710BD44
:102C64000009002001460148FFF754BF440000203A
:102C7400036803F01F020260034A04485B09012B46
:102C840008BF1046704700BF0028845000258450B8
:102C9400034B083033F81000C0F34010704700BFF6
:102CA4004800002070B50D4C00F1080334F81330CF
:102CB4000546DA050E4607D5C3F3432304EBC302E6
:102CC400526854F833309847A3682BB131462846EC
:102CD400E268BDE87040184770BD00BF480000209E
:102CE400124A083032F8103010B4D9051BD5C3F39A
:102CF400432123F4F85322F81030002002F1100489
:102D040034F8023B13F4807F03D0C3F34323994286
:102D140009D001303028F3D10023054810BC42F813
:102D24003130FFF719BF10BC704700BF48000020C6
:102D3400BC00002038B50246FFF7AAFF0B4C02F195
:102D4400080560B1002134F815305B0B9B0003F1DA
:102D5400A04303F55043C3F81015C3F810151046EB
:102D6400FFF7BEFF002324F8153038BD48000020CB
:102D74002DE9FF41044616461D4621B34E4F00F18E
:102D8400080837F818309B0706D5FFF781FF18B1FC
:102D94004A4804B0BDE8F08100232046CDE9003361
:102DA4008DF80E308DF80F300DF10F020B460DF13A
:102DB4000E0102F07BF837F8183023F0020343F0D9
:102DC400010327F8183096B13B483378726804F150
:102DD400080630F816108F070CD5002AD8D130F821
:102DE400162022F01C0242EA830320F81630CDBBE1
:102DF4003348CEE721F02001C904C90C20F816108D
:102E0400002AECD0032BC3D892F800C0624692008B
:102E140002F1A04202F5504223B9C2F81035C2F8BB
:102E24001035DCE7D2F8107541EA4C3127F003077E
:102E3400C2F81075D2F8107541F0200127F44F370D
:102E440027F44077C2F81075D2F810E5270207F48A
:102E54007C574EEA034E47EA0E07C2F8107520F875
:102E64001610BCE72046D5E90067FFF739FF002EAE
:102E7400BED0114D2B689E4204D16B689F4201D194
:102E840000220AE00F480DF10F01FFF743FE0C4B3F
:102E940098427FF47EAF9DF80F2005EBC2030834FF
:102EA4005F6035F8143045F8326043EA422343F456
:102EB400807325F814309BE7480000200400AD0B14
:102EC4000000AD0BBC000020F0B50446154685B0EB
:102ED40019B3344E00F1080736F81720930703D4CA
:102EE400FFF7D6FE00285AD112F01C0F02D04B78FF
:102EF400012B54D001238DF80F3000234A1CCDE957
:102F0400001320468B1C0DF10F0101F0CFFF36F8A2
:102F1400173043F0030326F8173015B9224805B0DB
:102F2400F0BD204E04F1080736F81700830736D5A4
:102F340095F800C00023614620F02000890001F1CB
:102F4400A041C00401F55041C00CC1F8103526F869
:102F54001700C1F810356A78002ADFD0D1F810358F
:102F6400AD7823F4991323F4F853C1F81035D1F84C
:102F740010E5230203F47C53120402F4403243EAC2
:102F84000E0313432A0502F4801240EA4C30134323
:102F940040F02000C1F8103526F81700BEE70348BA
:102FA400BDE700BF480000200000AD0B0400AD0BDE
:102FB400014BC3E9020170474800002008B50246EE
:102FC400FFF766FE38B1054B083233F81230044877
:102FD4005B0B0B7008BD0348FCE700BF48000020F2
:102FE4000000AD0B0400AD0B38B50F4C94F87850CD
:102FF400BDB96022294604F1100001F03AFC0D200D
:10300400FEF7A8F9094B0A48C3F87C51D3F87C2190
:103014004FF00042C3F80423012384F87830636737
:1030240038BD0448FCE700BF4800002000D0005031
:103034000000AD0B0500AD0B034B93F8780000388E
:1030440018BF0120704700BF480000200146014816
:10305400FFF782BDB800002001460148FFF75ABDC2
:10306400B800002037B50446FFF712FE1E4B04F1EA
:10307400080233F81230E8B113F002051AD15B0BE1
:103084009A0002F1A04000F5514002F1A04205600F
:1030940002F550420068D2F8100540F00100C2F871
:1030A400100529B1012202FA03F3104AC2F80433CD
:1030B40003B030BDC3F38203042B11D0052B11D010
:1030C40001A80194FFF7D4FD019B0169D94001F0E7
:1030D40001010231204603B0BDE8304001F02DBFAC
:1030E4000321F7E70221F5E74800002000D0005053
:1030F40008B50246FFF7CCFDC0B10F4B02F1080141
:1031040033F81130990711D401225B0B9A400B4913
:103114009B0003F1A043C1F8082303F55043D3F8FF
:10312400102522F00302C3F8102508BD0021BDE8D4
:103134000840104601F001BF4800002000D00050B4
:10314400104B00F1080233F8123013B5DB070446C4
:1031540016D5FFF7CDFF2046FFF7ECFD01A801943B
:10316400FFF786FD019B00EB8300D0F8003203F0EB
:10317400E04343F00203C0F80032034802B010BD3C
:103184000248FBE7480000200000AD0B0400AD0B33
:103194002DE9F04F002601223446604B6048614916
:1031A40087B01D6835B1D0F8045315421EBF1C60AA
:1031B4001D68164304338B424FEA4202F1D1DFF813
:1031C4006091D9F87C31002B00F08A80564F3B6A1D
:1031D40004933B62554B1A6A05921A624FF0000839
:1031E4000DF1100A4FEA4813009349E094FAA4F44D
:1031F400B4FA84F4009B4E4A1C4404F1080332F8E8
:103204001330E0089908C3F38205012304F0070290
:1032140003FA02FC1AF80020039422EA0C020AF8CA
:10322400002003A8FFF724FD039A4B0702F1800254
:1032340050F82220AB46C2F301422BD52046594612
:10324400D5B2FFF72FFD03A80394FFF711FD039BED
:10325400803350F82330C3F301439D4207D100214A
:10326400204601F06AFE2946204601F066FE03A8C6
:103274000394FFF7FDFC0122039B02FA03F30362AC
:103284005AF82840002CB1D1B8F1000F1AD14FF0F0
:103294000108A7E7022A0CBF03210221204601925C
:1032A40001F04BFE032D04D0019A022A06D1012D10
:1032B400DDD159462046FFF7F5FCD8E7032AD6D1DD
:1032C400022DF5E7C9F87C41D9F87C313A6A1749EF
:1032D40004923A620B6A05930B6213437FF47EAF48
:1032E400012416B907B0BDE8F08F96FAA6F3B3FA35
:1032F40083F304FA03F29B0003F1A04303F5504364
:10330400D3F81005D3F81015C0F30520C1F301411B
:1033140026EA0206FFF7C6FCE3E700BF00D100502F
:1033240000D0005020D10050002584500028845043
:10333400480000200E4B70B553F82040013053F87C
:103344002060A64200D870BDD4E9003528469847CD
:1033540065B1EB6830B10028B8BF4042FF28A8BF70
:10336400FF2018705A7842F001025A700834E8E7D6
:1033740088560000012208B5094B02201A70FFF795
:10338400D9FF00F051FF0320FFF7D4FF00F036F916
:10339400FDF74AF8034A137B23F00103137308BDB6
:1033A400190B00203002002008B50348034A00210D
:1033B400121A01F0F7FD08BD900100201C0B00203B
:1033C4000023012270B586B0CDE904230F220193B6
:1033D400CDE9023218234FF4A0720E4D0E4E03FBBA
:1033E40000550E4906EBC016044602FB00110C4BB7
:1033F4003046009500F0D2F8737B0A482C750134EE
:1034040023F0040300EBC4247373EE606C6006B015
:1034140070BD00BF08090020B0010020200F00206B
:10342400B93600006010002080B52D4BA6B003F51E
:10343400006282F3088883F30A880024E023294D7C
:10344400294E85F82230EC772C766C76AC7685F8AC
:1034540020406B6A254F43F4E0236B6285F82340D8
:10346400FEF758F9FDF758FF4FF0FF33AB62EB62FC
:10347400FEF760FBFEF7FEF940F20113ADF82430CD
:1034840006ABB360CDE91F44229401F065FD2046EC
:10349400FFF750FF0120164DFFF74CFF00F06CFCC6
:1034A400144BF5610593012313494FF48062CDE970
:1034B400034328463B46CDE90144009400F06EF8EE
:1034C40006466A7B284622F004026A7301F0FCFD7A
:1034D4002046FFF775FF3A4631462846FEF700F8C6
:1034E4006010002000ED00E008090020793300009E
:1034F40030020020E0570000200B002070B50E4B76
:103504000E4CA34201D3002070BDD3E9030141EA6C
:10351400000212F003020BD19D685A61AA4201D144
:103524001C33EEE75E6901320E6059610144F5E730
:103534006FF01500E8E700BF3C0100203C010020CB
:1035440037B50C464FF02005EFF3118185F312884F
:10355400BFF36F8F45695DB125602B684361836953
:1035640001338361002081F31188BFF36F8F11E071
:1035740052EA030C03D16FF00B002560F3E7CDE9A9
:1035840000230246083000F04DFB18B9024B9B683B
:103594005B69236003B030BD080900202DE9FF41B9
:1035A4000E9E00F1580506730426C0E91655002541
:1035B400044646730D9EC0E906558673D61D0C9AC3
:1035C40026F00706C0E919168560C573C566029220
:1035D4000B9A01EB060801920A9A00924246FDF703
:1035E40063FF054B65659B6803B11B6F404623670A
:1035F40004B0BDE8F08100BF080900202DE9F043C4
:10360400294C2A4D87B02646AE4204F130040FD32C
:1036140000F0C6F94FF4004640F2E737224CDFF8D9
:103624009090AC4220D307B0BDE8F04300F088BBD3
:1036340054F8043C54E90C01059354F8103C0493E9
:1036440054F8143C039354F8183C029354F81C3C6B
:10365400019354F8203C009354E90A23FFF79EFF9A
:1036640054F8303C5E65CEE7636A5A1C0DD00021E5
:10367400384623EAE373C3FB060151EAC333D4F8A3
:10368400008004D1404600F071FA3034C9E74FF4A9
:103694007A720023FCF75CFD02460B4608F1180021
:1036A400494600F0D3FCF0E73C0100203C01002037
:1036B400ED50000008B50B4C0B4D4FF02002EFF31A
:1036C400118382F31288BFF36F8F01F087FD2B788B
:1036D400A06113B9FDF726FEEFE7FDF76FFC0028A4
:1036E400EBD1F7E708090020190B00202DE9F3417D
:1036F400044617461E464FF02003EFF3118883F368
:103704001288BFF36F8FC368324A6BB180689168C7
:10371400884219D057EA060318D188F31188BFF3F9
:103724006F8F6FF00F000CE0916891F90E10013368
:10373400E36093682161A36088F31188BFF36F8FFE
:10374400002002B0BDE8F0812169F0E791F90E1084
:1037540090F90E306FF07E029942A8BF194691424B
:10376400B8BF11468B422EDD01F071FC054622469E
:103774004146CDE90076184800F054FA0028E0D01C
:103784004FF02003EFF3118683F31288BFF36F8F9A
:10379400236821699C420AD04BB193F90E309942B7
:1037A400A8BF19466FF07E039942B8BF1946A068B6
:1037B40001F04DFC00B945B13146074800F0DEF890
:1037C4006FF00A00BDE70025D1E786F31188BFF347
:1037D4006F8FF5E7080900201A0B002038B58368BD
:1037E4000446002B32D01C4A9268934231D1DA7BD2
:1037F400013ADA73C368012B05D9013BC36000F0B9
:103804009FFA002038BD4FF02003EFF3118583F3B6
:103814001288BFF36F8F0169806801F018FC20469D
:1038240001F0AEFCA06058B190F90E202261002294
:10383400826701F049FC2946084800F09FF8DEE75A
:10384400E06085F31188BFF36F8FD8E76FF0150040
:10385400D8E74FF0FF30D5E7080900201A0B002005
:1038640038B504464FF02003EFF3118583F3128833
:10387400BFF36F8F01F084FC48B10022826701F02E
:1038840023FC2946BDE83840044800F077B8D4E961
:1038940002329A4218BF0133A360F2E71A0B0020E8
:1038A40013B54FF02004EFF3118184F31288BFF3B2
:1038B4006F8F846844B1013C846081F31188BFF345
:1038C4006F8F002002B010BD52EA030406D181F3C9
:1038D4001188BFF36F8F6FF00F00F3E7CDE900237A
:1038E4000246024800F09EF9ECE700BF1A0B0020E4
:1038F40038B5074D2C6854B1FFF704F8054B044460
:103904001C6128680021BDE8384001F077BC38BD4F
:103914003809002008090020F8B504460D464FF088
:103924002003EFF3118783F31288BFF36F8F002115
:103934004FF4004C40F2E7300D4E002331614FF458
:103944007A72E4FB0C01FCF703FC002C094B0ADC43
:103954001860094BB0681D60FFF7CAFF87F3118830
:10396400BFF36F8FF8BD0228B8BF0220F0E700BF95
:1039740008090020380900203409002049B9EFF370
:10398400058030B9054BDA699B689A4201D0FDF78E
:1039940035BD81F31188BFF36F8F7047080900208C
:1039A4004FF02003EFF3118183F31288BFF36F8F7D
:1039B400044B9A68D37B013BD37381F31188BFF323
:1039C4006F8F70470809002038B502460C4801F093
:1039D40075FB0C4D044600B9EC68AB684AB95A7BD8
:1039E400D20606D1A26922B9DA897F2A01D9EB610C
:1039F40038BD9C4202D02046FFF77AFFEC61F7E71E
:103A0400280900200809002070B590F90D2001460E
:103A1400002A437B04DA03F07F03437301F026FB9F
:103A24004B7B154A63F07F034B7302F12005D2E907
:103A34000834AB421BD0D3B191F90E6093F90E0058
:103A440086420FD0801B00280CDD5868C1E9003085
:103A5400016059609068BDE87040431A584258416B
:103A6400FFF7B2BFA34202D01B68002BE6D1C1E925
:103A7400005421605162EDE70809002038B54FF089
:103A84002003EFF3118583F31288BFF36F8F174B75
:103A9400174A9C6811688C4207D12046FFF728FF1B
:103AA40085F31188BFF36F8F38BD00211160114A6F
:103AB4001268C2B1E2897F2A15D8627BD20612D17C
:103AC4000D4A94F90E10126891420CDB0B4A944291
:103AD40009D01A69824203DC2046FFF795FFDCE730
:103AE400121A1A61DCE70022FBE700BF0809002074
:103AF400300900203809002034090020B0010020DA
:103B040070B490F90D20437B002A2ADBDA0628D111
:103B1400826932BB144A63F07F03437302F12005C8
:103B2400D2E90834AB4217D0B3B190F90E6093F9DF
:103B34000E108E420BD0891B002908DD5A68C0E99B
:103B4400003210605860002070BCFFF73DBFA342F4
:103B540002D01B68002BEAD1C0E9005420605062F7
:103B6400F1E770BC704700BF0809002010B54FF0A2
:103B74002002EFF3118482F31288BFF36F8F427B2C
:103B8400510704D484F31188BFF36F8F10BD22F062
:103B940004024273FFF7B4FF2146BDE81040014818
:103BA400FFF7ECBE1A0B002008B590F90D20014672
:103BB400002A437B04DA03F07F03437301F056FACF
:103BC400044B9868431A58425841BDE80840FFF72F
:103BD400FBBE00BF080900202DE9F041064615464A
:103BE4001C464FF02003EFF3118783F31288BFF3D1
:103BF4006F8F01F09BFA87F31188BFF36F8FB4F1D5
:103C0400FF3F08BFB5F1FF3F08D02A46234606F11F
:103C140018000349BDE8F04100F018BABDE8F0818E
:103C2400ED50000010B50C46064B11469868064B43
:103C34001860DDE90223FFF7CFFF2046BDE81040FE
:103C4400FDF7DCBB0809002030090020F8B5044664
:103C54004FF02003EFF3118683F31288BFF36F8FC5
:103C6400437B49B2DA0633D182698ABB03F07F030E
:103C7400437301F0FBF9437B174A63F07F034373FB
:103C84008173104650F8203F83421BD0D3B1576A4A
:103C940093F90E50A94210D06D1A002D0DDD5A680B
:103CA400C4E9003214605C600120FFF78DFE01203E
:103CB40086F31188BFF36F8FF8BDBB4202D01B6837
:103CC400002BE5D1536AC4E900031C605462EBE79E
:103CD4000020A173ECE700BF0809002070B504467A
:103CE400183001F065FA4FF02003EFF3118683F3E7
:103CF4001288BFF36F8F94F90D20637B002A05DAD5
:103D040003F07F032046637301F0B0F90B4D637B2E
:103D1400A86843F010036373031B58425841FFF72C
:103D240053FE86F31188BFF36F8FAB68A34203D1B0
:103D3400BDE8704001F0B8B970BD00BF08090020AB
:103D440010B54FF02003EFF3118483F31288BFF30F
:103D54006F8F084B00209A68D37B0133D373FFF72E
:103D640033FE84F31188BFF36F8FBDE8104001F078
:103D74009BB900BF080900200021044B084603F149
:103D84002002C3E90822FFF7C7BD00BF08090020CD
:103D9400F8B54FF02003EFF3118583F31288BFF3D6
:103DA4006F8F1A498868437B03F07F03437301F0E4
:103DB4005DF908468B685A7B62F07F025A7350F8AB
:103DC400202F82421CD0DAB14F6A93F90E6092F927
:103DD4000E40A6420FD0A41B002C0CDD5168C3E991
:103DE40000210B6053600120FFF7EEFD2846BDE87B
:103DF400F840FDF703BBBA4202D01268002AE6D1AC
:103E04004A6AC3E9000213604B62ECE70809002028
:103E140050EA01032DE9F04105460E4603D1FFF7B0
:103E2400B7FF002033E06FF001044FF0FF33241A92
:103E340063EB0103012C73F1000302DA01F0F8F9DA
:103E440044194FF02003EFF3118883F31288BFF372
:103E54006F8F104F104BB8681860FFF7A5FEB86855
:103E64000E492A463346183000F0F0F8BA68404646
:103E7400537B43F010035373FDF7C0FA01F0D8F9F4
:103E8400201A63EB0303012873F10003C9DBBDE8C7
:103E9400F08100BF0809002030090020ED50000027
:103EA400B1F1FF3F08BFB0F1FF3F08B506D1084BA1
:103EB4009868FFF713FF4FF0FF3008BDFFF7A8FF26
:103EC4004FF47A7380FB0303C00B40EA4340F4E7EA
:103ED40008090020014B9868704700BF08090020BA
:103EE4002DE9F04104464FF02003EFF3118683F3EC
:103EF4001288BFF36F8F437B1A0705D586F31188A9
:103F0400BFF36F8FBDE8F08123F0200242F0080177
:103F1400D20920D14173A36813B1204601F0AEF851
:103F240004F1180001F044F94FF0000804F15807B7
:103F3400A56DBD4200D0B5B90120FFF745FD104B7A
:103F44009B68A342DAD1EFF30583002BD6D1304628
:103F5400FDF754FAD2E703F05F0343F00803437319
:103F640001F084F8D7E7284601F088F805F1180035
:103F740001F01EF92846C5F87880FFF7C1FDD7E7A0
:103F84000809002008B50648064A0749121A01F034
:103F94000BF8BDE80840054A0549064801F004B895
:103FA400000000208C0100201C58000000000000CC
:103FB4001C58000000000020034B1B680BB9FEF7DF
:103FC400A1BC0020704700BF3C090020104B10B575
:103FD4001C689C4208BF0024FFF7EEFFA4B1D4E99B
:103FE40004321B1A62EBE070B3F1004F70F100026F
:103FF4000ADA0028ACBF18460020064B1B6913B12F
:104004009842A8BF184610BD6FF00040F5E700BF06
:10401400C40000200809002030B5036868B10A4ACA
:104024005268904209D043B1D3E90421D0E9044550
:10403400121941EB0501C3E90421426813605A6077
:104044000023C0E9003330BDC4000020B3F1FF3FBA
:1040540008BFB2F1FF3FF8B504461F46154667D0C6
:1040640081604FF02003EFF3118683F31288BFF3CE
:104074006F8F6FF001024FF0FF3C531B6CEB070393
:10408400002B1BDB2B4BD3E90013521A6CEB0303FD
:10409400551B63EB0703012D73F10002BCBF01251F
:1040A4000023C0E904532448D0E9003C834218D1DA
:1040B400C4E9000CCCF80040446026E0FFF77CFF24
:1040C400013547F100072D1847EBE077C4E90457A1
:1040D400E9E7521A65EB07059C45C4E90425E7D0D6
:1040E4001B68002BE4D0D3E90417D4E904258A42E1
:1040F40075EB070EEDDA8A1A67EB0505C3E90425AB
:104104005A68C4E9003214605C60036883420BD0CF
:104114009C4209D1FFF75AFF18B1084B1B6983422F
:1041240002D00021FEF7BEFB86F31188BFF36F8F28
:10413400F8BD00BFB0020020C40000200809002020
:104144002DE9F8430546FFF799FC4FF02003EFF300
:10415400118483F31288BFF36F8F244EDFF89080AD
:104164003560244DD8F80000326840454FEAE277C4
:10417400D5E9001E0BD050B1D0E9043C9A4277EB4C
:104184000C0916DA9B1A6CEB070CC0E9043C5218B4
:104194004EEB0707C5E9002700253560FFF716FF3A
:1041A4002946FEF77FFB84F31188BFF36F8FBDE8C8
:1041B400F88359184EEBE377D31A336000220023B7
:1041C400C0E90423C5E90017FFF726FF84F311882B
:1041D400BFF36F8F836898474FF02003EFF3118488
:1041E40083F31288BFF36F8FBCE700BF3C09002044
:1041F400C4000020B002002010B54FF02003EFF3FC
:10420400118483F31288BFF36F8FFEF77BFB054A9B
:10421400D2E90031C01841F1000184F31188BFF3E1
:104224006F8F10BDB0020020024A0349034800F01A
:10423400A1B900BF18580000E5570000F25700006C
:1042440010B50A4C23681BB101230020236010BD64
:1042540000F0DCF80028F7D00138072803D8044B15
:1042640053F8200010BD034810BD00BF40090020D2
:10427400A0560000FE8FFFFFBFF34F8F0549064B8A
:10428400CA6802F4E0621343CB60BFF34F8F00BFF0
:10429400FDE700BF00ED00E00400FA0530B44FF084
:1042A400FE3200250B4B0C4C0C494968C3F8002422
:1042B400C3F80424C3F80824C3F80C24C3F8102456
:1042C400C3F81424C3F81824C3F81C24C4F80055F4
:1042D40030BC08470050845000408450CC0000207B
:1042E400024BD0E90012C3E900127047CC00002051
:1042F40010B5044630B16368DB0602D500232360A1
:10430400636010BD024B03485B689847F3E700BF46
:10431400CC000020C0560000B0B1436893B1DB0666
:104324000ED5012350E8002F194640E8001C9CF0EC
:10433400000FF7D1012AF5D0BFF35F8F002070473B
:1043440003487047034870476FF4E040704700BF6C
:10435400E98FFFFFEA8FFFFF034668B142683AB175
:10436400D20607D5BFF35F8F002210461A6070474C
:1043740003487047034870476FF4E040704700BF3C
:10438400EA8FFFFFE98FFFFF10B5044620B100223A
:1043940011232260636010BD0148FFF77FFFF6E739
:1043A400E856000070B5164CD0F804C00668C4F88E
:1043B40004C0D0F808C0C068C4F808C0E060266033
:1043C4000868104B104D18604868D5F818215860DB
:1043D40088689860C8680969D8601961D3060DD5E2
:1043E400002305F58A70C5E94533C5E96E33B04746
:1043F400236805F5DC70BDE87040184770BD00BF48
:10440400DC000020EC0000205809002008B500F072
:1044140011F830B900F010F838B9054AC2F80C0A9E
:1044240008BD00F037F8032008BD042008BD00BF14
:10443400005084500020704710B5114800F048F82F
:1044440000B110BD0F4800F043F80028F9D10E4C1C
:10445400204600F03DF80028F3D10C4B0C481C60BA
:1044640000F036F801460028EBD100F02DF80446A0
:1044740008B1204610BD00F03FF82046FAE700BF1F
:104484002401002018010020200100202801002020
:104494001C01002008B5084800F024F8074800F083
:1044A40021F8074800F01EF8064800F01BF8BDE8A4
:1044B400084000F00BB800BF2401002018010020C0
:1044C400200100201C01002000207047704700BF1D
:1044D40008B5034B02681B6810689847002008BDA4
:1044E400DC00002008B5034B02685B68106898473D
:1044F400002008BDDC00002070B5094C094D20697E
:10450400AB68984718B1084B08485B689847002186
:10451400074AEB6811602069BDE87040184700BF86
:10452400EC000020DC000020CC0000200C57000030
:1045340054090020034658B1426802F00302012ADC
:1045440003D0032A04D1026812B100209860704796
:104554006FF0150070474268034602F00302032A15
:104564004FF00002816014BF104600685A60704723
:10457400002070470FB407B504A951F8040B01914A
:10458400FBF786FF03B05DF804EB04B07047038BC0
:1045940013F0070305D10368002B0CBF0020032090
:1045A4007047022B05D1438B002B14BF002004203D
:1045B4007047012B05D10368002B0CBF0020052098
:1045C4007047002070472DE9F0410D460746194613
:1045D400281D90461E46FFF7BEFF044638B13346F9
:1045E400424629463846A446BDE8F0416047BDE846
:1045F400F08110B44FF02004EFF3118284F3128899
:10460400BFF36F8F416110BC0121FBF74FBF10B5A1
:104614000C4640B139B1081DFFF78CFF28B9A368D7
:1046240033F0030301D06FF0150010BD38B50C460C
:10463400054658B151B10B6843B14B6833B11C22E4
:10464400002100F016F900202C6138BD6FF0150030
:10465400FBE770B504460E46FFF7D9FF051E31DBB4
:104664004FF02003EFF3118183F31288BFF36F8FB0
:104674004FF6FF75638B208BAB4200F007022ED000
:10468400022A0ED1013363831546012381F3118875
:10469400BFF36F8FB3B1002331462046FFF793FF7A
:1046A40010E0830701D0062A0ED10023336063682B
:1046B40093B9C4E90066154662B90A462046022148
:1046C400FBF7F4FE284670BD052A0CBF6FF0850584
:1046D4006FF004050023D9E71E606660EBE76FF016
:1046E4000A05F7E7044608B5084611461A46A047E6
:1046F400FFF7F0FBFDF7A8F82DE9F84F9A46D378B9
:1047040080466F2B0F461546A3F1410B29D024D8C0
:10471400582B14BF0A261026DDF8289032460023B1
:1047240040463946FBF714FD092AD4B21ED830346A
:10473400B045E4B277F1000309F8014D01D3D14546
:1047440011D82B789B0605D5082E15D1AB7843F0EC
:104754000803AB704846BDE8F88F03F0F703702BED
:10476400D7E70826D8E780460F46D7E7BBF1190FED
:1047740094BF37345734DBE7102EEBD1AB7843F0DA
:104784001003E6E72DE9F0410746884615461E4624
:104794001446B442A4EB050002D33EB923782BB1EE
:1047A400414614F8010BB8470028F2DABDE8F0815D
:1047B4007047002383F31188BFF36F8F7047002085
:1047C40008B5FCF715FB00F0D2BB0146006800F009
:1047D400CEBB00210120FFF7F6BF08B5FCF7EEFDC4
:1047E400BDE80840FCF7B0BE436E83F30B88704706
:1047F40040E800F313F4803FD8B208BF6FF015000F
:1048040070477FB50A894E890B684D6802F01F0214
:1048140042EA461200938DF8082023F01F036A1E13
:10482400134423F01F030728039304D86946FDF7B4
:104834003DF804B070BD6FF01500FAE703460020A0
:104844001A5C02B970470130FAE7034600201A5C8B
:104854000AB1884200D170470130F8E710B5431E11
:104864000A44914200D110BD11F8014B03F8014FE5
:10487400F7E70346C9B20244934200D1704703F8F4
:10488400011BF9E74FF0FF3070470C220369C9B2EE
:1048940001FB0233986F00F0070070474FF02003CC
:1048A400EFF3118283F31288BFF36F8F036803F071
:1048B400C00343F00203036082F31188BFF36F8FD8
:1048C4007047034670B50069C9B24FF02004EFF396
:1048D400118684F31288BFF36F8F0C2505FB010446
:1048E400A46F14F0C00401D0A24210D1012205FB30
:1048F40001008267002086F31188BFF36F8F28B907
:104904005B6803EBC1014B689847002070BD4FF012
:10491400FF30F0E78022FFF7D4BFF8B5069F0546C5
:104924000469C9B24FF02000EFF3118C80F31288B0
:10493400BFF36F8F0C2606FB0146B06F00F0070E25
:10494400BEF1010F11D1B76700268CF31188BFF3B4
:104954006F8F46B90C2000FB0144C4E91C236B682B
:1049640053F8313098473046F8BD00F0C000874214
:1049740014BF4FF0FF366FF07706E6E713B58024D7
:104984000094FFF7CAFF02B010BD10B41C240069E4
:10499400CBB203FB0400002110BC1047032000F03D
:1049A40023BA022000F020BA002000F01DBA032030
:1049B40000F07ABA022000F077BA002000F074BA4E
:1049C4001046FEF74DBF436800205B681B690B600F
:1049D400704743685B68586842400A4042405A60E6
:1049E40000207047436800205B6899607047436803
:1049F40000205B68D9607047436800205A68536898
:104A04004B4053607047036930B5586858B100246F
:104A1400814212D108689D6854B98D42586000D112
:104A24009860002008606AB9002030BD2846EFE78E
:104A34008D42206008BF9C60F3E705680446002DA2
:104A4400F4D13AB15A6898680A6059600028EBD1E9
:104A54009960EAE76FF01500E7E70B460269D2E9CF
:104A6400010183E803000020704743681B68D3F802
:104A74008004C3F880047047436802691B68D3F854
:104A8400100148B10020527C0A70C3F81001D3F819
:104A9400102101221A6070474FF0FF3070470268FE
:104AA4000346D2F8580140B95B689B0706D4D2F894
:104AB4002001003818BF0120704701207047426868
:104AC4001368D3F80413C90518D5D3F82011A9B174
:104AD4004FF02000EFF3118180F31288BFF36F8F42
:104AE400D3F8200130B10020C3F82001D3F820010D
:104AF4000120D86081F31188BFF36F8F5268D2060A
:104B040015D54FF02001EFF3118281F31288BFF322
:104B14006F8FD3F8581111B10021C3F800154FF469
:104B24008001C3F8081382F31188BFF36F8F7047B5
:104B3400704730B543681360037A03F10053013BB7
:104B4400DB00456814681D44AC4202D96FF00100D3
:104B540030BD65798D4202D008341460F1E700203D
:104B6400F6E709B9FDF7D8BEFDF70EBF70B51546D7
:104B7400044600EB8106A64201D1002070BD2368E3
:104B84001A0C222A00F28E80DFE802F0121D244360
:104B94002939438C8C8C8C484D8C8C8C8C8C8C8CD3
:104BA4008C8C525E63688C8C8C6D73787D828700EC
:104BB40003F03F03C5F80C35206800F03F00FDF713
:104BC400E3FE012215E003F03F03C5F8143500228B
:104BD40000210FE003F03F03C5F80835ECE703F0CC
:104BE4003F03C5F80835206800F03F00FDF794FE48
:104BF400002201212068FDF79FFE0434BBE703F087
:104C04003F03C5F80C35206800F03F00FDF784FE33
:104C1400D7E703F03F03C5F81035D8E703F03F03A7
:104C2400C5F80835D3E703F03F03C5F80C35CEE7E4
:104C340003F03F03C5F860352068C0F3403100F04D
:104C44003F00FFF78EFFBCE703F03F03C5F8643570
:104C5400F2E703F03F03C5F86835EDE703F03F03DF
:104C6400C5F86C35E8E703F03F03C5F824350122A5
:104C7400AEE703F03F03C5F82835F8E703F03F0338
:104C8400C5F83035F3E703F03F03C5F83435EEE7F4
:104C940003F03F03C5F83835E9E703F03F03C5F8EF
:104CA4003C35E4E76FF0850068E7002008B5FCF7C1
:104CB40083FDFFF7C5BA08B5FCF752FAFCF716FBFB
:104CC400BDE80840FFF7BCBA004700F0B5BAF7B535
:104CD4000546032874D8DFE800F002212D3B4FF08D
:104CE40050230222C3F808230022C3F80421D3F876
:104CF40004210122DA6001239D4218BF002442F2FC
:104D040010774FF050268DF8073008BF0DF10704D7
:104D1400032D55D8DFE805F02A3B444D4FF05023CE
:104D240001220021C3F80823C3F80011D3F80011AD
:104D34005A60E0E74FF050234FF40072C3F80823A1
:104D44000022C3F82421D3F8242101225A62D2E795
:104D54004FF050234FF48072C3F808230022C3F8A5
:104D64002021D3F820210122DA61C4E724B1D6F846
:104D7400183403F003032370D6F81834DB031FD56B
:104D8400D4B90120FFF7A1FF013FC1D118E024B13C
:104D9400D6F80C3403F001032370D6F80C34EDE795
:104DA40024B1D6F85C3403F001032370D6F85C34E4
:104DB400E4E7D6F85434E1E79DF80730012BE0D05E
:104DC40003B0F0BD08B50520FCF7D4FA10B90520EE
:104DD400FCF7C0FA4FF050230122C3F81825C3F89A
:104DE4001425C3F8802508BD08B503281ED8DFE8BC
:104DF40000F002333F4D4FF05022D2F81834D2F86D
:104E04001814C90313D4D2F81434DB0719D40123BA
:104E14004FF05022C2F818350023C2F80431D2F8FA
:104E240004310223C2F804330123936008BD03F064
:104E34000303022BECD0012BEAD00020FFF747FF3D
:104E4400E5E7D2F81C3403F00303013B012BF4D84B
:104E54000223C2F80433E9E74FF050230022C3F8D9
:104E64000021D3F800210122C3F804231A60DDE7EE
:104E74004FF050230022C3F82421D3F824214FF407
:104E84000072C3F8042301221A62CFE74FF05023C3
:104E94000022C3F82021D3F820214FF48072C3F8F4
:104EA400042301229A61C1E7FFF711BFF7B5174642
:104EB400DDE90846019001A81D46FDF7D9FE019BD6
:104EC400002F00EB830014BF02230023002918BF26
:104ED40043F00103002D14BF4FF00C0C4FF0000CF5
:104EE400002C43EA0C0314BF4FF4706C4FF0000C19
:104EF400002E43EA0C0314BF4FF4403C4FF0000C67
:104F0400D0F8002243EA0C0322EA030301B1097832
:104F14000FB13F787F0019430DB12D78AD003943AF
:104F24000CB1227814020D430EB1367836042C43AA
:104F34003443C0F8004203B0F0BD1FB50DF10F03B8
:104F4400019300238DF80F101A4619460093FFF7BA
:104F5400ADFF05B05DF804FB704738B1C36818882D
:104F6400C0F30800A0F58073584258417047F8B563
:104F740005460E464FF02003EFF3118783F31288A2
:104F8400BFF36F8FFEF7A6FF314604462846FFF7AE
:104F94008CFE87F31188BFF36F8F2046BDE8F8407D
:104FA400FCF752BCFFF765BCFFF758BC30B50024D2
:104FB400846141EA020414F00304C0E9023201618D
:104FC4000CD14461A34203D1C0E90000002030BDEC
:104FD400456901340D6041611144F3E76FF0150038
:104FE400F5E7F8B504460D464FF02003EFF31186BC
:104FF40083F31288BFF36F8F476977B900F0C0F865
:1050040058B12A688767426100F05EF8314604F1BE
:105014000800BDE8F840FEF7B1BC2B6862691A606D
:105024002B686361A369013BA36186F31188BFF315
:105034006F8FF8BDEFF30580003818BF012070476B
:1050440008B5FBF781FFBDE80840FFF771BD90F993
:105054000E308B4201D0FEF7F9BD002070470346A5
:105064000020C3E90033C3E902007047D0E90032ED
:1050740013605A600023C0E90033704708B5FFF796
:10508400F5FF437B23F0020343730023836008BDD1
:10509400034620B9EFF305820AB9FCF7AFB983F3ED
:1050A4001188BFF36F8F70474FF02003EFF3118027
:1050B40083F31288BFF36F8FFFF7EABF03460068DC
:1050C400834208BF0020704710B54FF02003EFF370
:1050D400118483F31288BFF36F8FFEF711FD84F3FD
:1050E4001188BFF36F8F10BD014610B54FF0200338
:1050F400EFF3118483F31288BFF36F8F10F80B3C26
:1051040013F0280F0DD151F8103C18380BB1FFF7EC
:10511400B5FF11F80B3C23F0140301F80B3CFEF728
:10512400EFFC84F31188BFF36F8F10BD38B50446CC
:105134000D46FEF739FD637B43F00203637395B1BB
:105144002B68A5609D4215D0A3B194F90E1093F974
:105154000E20914208D0521A002A05DD5A68C4E98B
:10516400003214605C6038BD6A68934202D01B68E8
:10517400002BECD16B68C4E900531C606C60F2E74F
:1051840038B54FF02003EFF3118583F31288BFF392
:105194006F8FFFF793FF044620B1FFF76FFF1830BE
:1051A40000F006F885F31188BFF36F8F204638BDF1
:1051B40010B54FF02002EFF3118482F31288BFF38D
:1051C4006F8F03683BB1FEF727FF002084F311883B
:1051D400BFF36F8F10BD6FF01500F7E710B54FF0F8
:1051E4002003EFF3118483F31288BFF36F8FFEF76C
:1051F400EDFE84F31188BFF36F8F10BD70B50446C4
:105204000D464FF02003EFF3118683F31288BFF3AA
:105214006F8FFEF7DBFE012805DDA04203DB294684
:105224002046FDF73FFB86F31188BFF36F8F70BDF7
:1052340008B5FEF7E1FF08BD08B1FBF723BE7047D0
:0852440070470000FDF7D2BB2A
:08524C003CAFFF7F01000000F0
:10525400390E000000000000051C0000A4520000EC
:105264000135000000000000B51F0000D45200000A
:10527400B51F0000BC520000B74C00000000000045
:1052840001230000EC520000851E00000000000015
:105294004127000000000000BB4C0000000000009B
:1052A400BD570000D0550000B85500002C01002067
:1052B400300800203E550000CA5700002056000068
:1052C400FC55000034010020DC08002038550000A3
:1052D400C357000030560000FC5500003001002088
:1052E400E808002032550000D1570000785600002D
:1052F40064560000380100202C0000202C550000CA
:1053040000000000D747000000000000D74700005D
:1053140000000000D747000000000000D74700004D
:1053240000000000D7470000B92B0000CD4C00005E
:1053340000000000D747000000000000D74700002D
:10534400EC520000C34A000000000000D7470000F0
:1053540000000000D747000000000000D74700000D
:1053640000000000D747000095310000CD4C00003C
:1053740000000000D747000000000000D7470000ED
:1053840000000000D747000000000000D7470000DD
:1053940000000000D747000000000000D7470000CD
:1053A40000000000D747000000000000C1270000F3
:1053B40000000000D747000000000000D7470000AD
:1053C40000000000D747000000000000D74700009D
:1053D40000000000D747000000000000D74700008D
:1053E40000000000D747000000000000D74700007D
:1053F40000000000D747000000000000D74700006D
:1054040000000000D747000000000000D74700005C
:1054140000000000D747000000000000D74700004C
:1054240000000000D747000000000000D74700003C
:1054340000000000D747000000000000D74700002C
:1054440000000000D747000000000000D74700001C
:1054540000000000D747000000000000D74700000C
:1054640000000000D747000000000000D7470000FC
:1054740000000000D747000000000000D7470000EC
:1054840000000000D747000000000000D7470000DC
:1054940000000000D747000000000000D7470000CC
:1054A40000000000D747000000000000D7470000BC
:1054B40000000000D747000000000000D7470000AC
:1054C40000000000D747000000000000D74700009C
:1054D40000000000D747000000000000D74700008C
:1054E40000000000D747000000000000D74700007C
:1054F40000000000D747000000000000D74700006C
:1055040000000000D747000000000000D74700005B
:1055140000000000D747000000000000D74700004B
:0855240000000000D747000061
:10552C0000800080FF7F00800080FF7F0080008073
:08553C00FF7F00800080FF7F6B
:0C554400FFFFFFFFFFFFFFFFFFFFFFFF67
:105550000338FDD87047000000000000C34700007A
:105560008112000071110000B91100002112000029
:10557000200000200800002018000020000000008B
:1055800010000020000000200000000006000100C4
:10559000020000009855000000000000AE57000017
:1055A00006000000E0FF0F0000000020B6570000DA
:1055B00021000000E0FF0620311D00001949000015
:1055C00081490000000000008F480000000000003A
:1055D000CD1C0000651D0000AD490000BF49000062
:1055E000A7490000B9490000A1490000B3490000E3
:1055F000C11B0000911B00000000000031200000D2
:10560000CB490000D7490000E9490000F3490000F8
:10561000FD490000DD1E00000B4A000000000000F4
:10562000FFFFFFFF00258450000000000000000085
:10563000FFFF00000028845000000000010000006F
:10564000008000505C5600000100000014000000C3
:1056500013000200D6000100D50003004C560000E4
:10566000040000007D4A0000F12300006F4A0000A2
:10567000852100005F4A0000008000500200000009
:1056800000000000405600005452000094520000F8
:105690009C520000A4520000A4520000F5FFFFFF3E
:1056A000FF8FFFFFFF8FFFFFFE8FFFFFFE8FFFFFCC
:1056B000FD8FFFFFFC8FFFFFFC8FFFFFFB8FFFFFC6
:1056C0006D757465785F667265652063616C6C6585
:1056D000642077697468204E554C4C20706172616B
:1056E0006D6574657200000043616E277420696EF9
:1056F000697469616C697A65206D757465782C20B0
:10570000776173204E554C4C0D0A0000436F756C49
:1057100064206E6F74206C6F636B20706F7765729E
:105720002073617665206D7574657800286E696CEC
:1057300029004661696C656420746F207265626F30
:105740006F743A207370696E6E696E6720656E645F
:105750006C6573736C792E2E2E0A006D75746578E6
:105760005F696E69742063616C6C6564207769742D
:1057700068204E554C4C20706172616D6574657285
:1057800000436F756C64206E6F7420616C6C6F6386
:10579000617465206D75746578206265666F7265E9
:1057A00020696E697469616C697A696E6700464C3C
:1057B0004153485F30005352414D5F3000434C4FDE
:1057C000434B004750494F5F31004750494F5F30CE
:1057D00000554152545F30000100000001010000FB
:1057E0006D61696E0076332E302E39392D6E6373FC
:1057F00031002A2A2A20426F6F74696E67205A6529
:1058000070687972204F53206275696C642025732B
:0C581000202573202A2A2A0A000000002C
:10581C0075450000FFFFFFFF3C0100200100000068
:10582C005001002001000000640100200100000074
:10583C0078010020010000008948000000000000F1
:10584C0000C2010000010300000000000000000085
:10585C000090D003FFFFFFFF0000000000000000DD
:10586C00000000000000000000000000000000002C
:10587C00000000000000000000000000000000001C
:10588C00000000000000000000000000000000000C
:10589C0000000000000000000000000000000000FC
:1058AC0000000000000000000000000000000000EC
:1058BC0000000000000000000000000000000000DC
:1058CC000000000000000000FF00000000000000CD
:1058DC0000000000C4000020C400002000000000F4
:1058EC007D42000044090020110000008D4300009F
:1058FC00F54200001D4300005D4300001001002034
:10590C00D40000200801002000000000000100204D
:10591C0048090020110000004C0900201100000073
:10592C005009002011000000F0000020FC000020B5
:0C593C00F4000020EC00002020010020FE
:10594800000000000000000000000000000000004F
:105958003C0100203C010020000000000000000085
:105968000E0000005001002050010020000000003F
:10597800000000000E000000640100206401002007
:1059880000000000000000000E0000007801002068
:105998007801002000000000000000000E00000058
:040000030000175D85
:00000001FF
